:100000000EC028C027C026C025C024C023C022C0DF
:1000100021C020C0B2C01EC01DC01CC01BC0112406
:100020001FBECFE5D1E0DEBFCDBF10E0A0E6B0E05F
:10003000E0E3F3E002C005900D92A236B107D9F7D4
:1000400020E0A2E6B0E001C01D92A836B207E1F7B9
:10005000EED06CC1D5CF861718F0861B869502C0EE
:10006000681B6695860F089590916400913001F1A8
:1000700060916500861718F0982F961B02C0962F86
:10008000981B9233A8F0E7DF91E090936400909181
:100090006700981710F0981B03C0282F291B922F78
:1000A0009A3130F080936700682F80E090E02CC197
:1000B00008953D9A379A86B1836086B9089597B1BD
:1000C000907E8F71892B87B9369A3699FECF84B18D
:1000D00085B10895FF920F931F93CF93DF93F82E6E
:1000E000D62FC0E000E010E0CD1731F08F2DE7DF14
:1000F000080F111DCF5FF8CF6C2F70E0C801E8D05A
:10010000862FDF91CF911F910F91FF900895009757
:1001100041F0E9EFF0E03197F1F700C000000197FE
:10012000F6CF0895CF9363E083E0D4DFC82F9CDF40
:100130009091670081E0B49903C09C1720F402C03D
:100140009C1708F080E0CF910895CF93C5E683EC2B
:1001500099E00197F1F700C00000E4DF90916000A2
:10016000891731F081E0892780936000C1E002C0E7
:10017000C15069F78C2FCF9108951F920F920FB63F
:100180000F9211242F933F934F935F936F937F931D
:100190008F939F93AF93BF93EF93FF9388B3897F20
:1001A00088BB8091620090916300019690936300F8
:1001B00080936200803B944029F4809166008130F6
:1001C00009F4C19A8091620090916300823B94404F
:1001D00049F480916600813009F4C19A109263005D
:1001E000109262009FDF813011F4C09A0FC0C09856
:1001F00080916600813051F480916200909163009B
:1002000065E070E065D0892B09F4C29AFF91EF9107
:10021000BF91AF919F918F917F916F915F914F911E
:100220003F912F910F900FBE0F901F90189587B39D
:10023000876087BB88B3887F88BB87B3877E87BB8F
:10024000C49AC3988AB582608ABD83B7856083BF2C
:1002500089B7806189BF82E689BD80ED97E057DF6D
:1002600028DF63E083E036DF80936500789480E0E8
:1002700090E042D08093670081E090E03DD0809391
:10028000660080916600823018F081E080936600FD
:10029000C0E0D1E05ADF882311F0CF5F01C0C0E099
:1002A00080916600813011F4C63031F08091660093
:1002B0008111F0CFC33071F7809166008D27809354
:1002C00066006091660081E090E01ED0C0E0E2CF61
:1002D000AA1BBB1B51E107C0AA1FBB1FA617B7076C
:1002E00010F0A61BB70B881F991F5A95A9F7809588
:1002F0009095BC01CD010895E199FECF1FBA8EBB48
:10030000E09A99278DB30895262FE199FECF1FBA61
:100310008EBBE09A81500DB2021639F01CBA2DBB8B
:100320000FB6F894E29AE19A0FBE0895F894FFCFC1
:020330000100CA
:00000001FF
